:103C000005C001C0089581E05AC0089580E057C002
:103C100008958CE089B910BC82E08BB986E880BD3C
:103C200088E18AB908955D9BFECF8CB90895A8EB11
:103C3000BBE01197F1F70197D1F7089580E090E08C
:103C40005F9B02C081E090E008955F9BFECF8CB146
:103C500099270895FADF803221F484E1E4DF80E1DE
:103C6000E2DF0895CF93C82FF0DF803231F484E192
:103C7000DADF8C2FD8DF80E1D6DFCF9108951F9354
:103C8000CF93182FC0E0C81720F4DFDFCF5FC11734
:103C9000E0F3CF911F9108952FB7E199FECF9FBB1D
:103CA0008EBB6DBBF894E29AE19A2FBF0895E1991B
:103CB000FECF9FBB8EBBE09A8DB399270895CC248D
:103CC000DD247601C82FF89411248EE58DBF84E0A1
:103CD0008EBF9FDFC69ABC9ACC2329F084E1A3DF74
:103CE00080E1A1DF25C08C2F9EDF1C2FE0E0F0E0FB
:103CF00084918F3F39F0B69B05C011E0CEE103C03F
:103D0000A9DF16C0C6E0C150CF3F71F084E690E055
:103D10008EDF88B390E1892788BB90DF882399F3F1
:103D200094DF803369F3EFCF112311F00C9400007E
:103D3000C49A8BDF803309F44FC08133A1F485DF4F
:103D4000C82F8032B1F784E16EDF81E46CDF86E555
:103D50006ADF82E568DF8C2F66DF83E564DF84E558
:103D600062DF8BE4DDC0803429F46FDF8638A0F198
:103D70006CDF32C0813491F468DF803811F482E066
:103D8000D7C0813811F481E0D3C0823811F482E1C8
:103D9000CFC0883909F0CBC083E0CAC0823411F4A7
:103DA00084E103C0853419F485E069DF15C08035EE
:103DB00011F0823511F4C4980FC0813539F4C49ADA
:103DC00049DF82E090E033DF1BDFB3CF853531F48C
:103DD0003CDFC82E3ADFD82E3DDFABCF863519F455
:103DE00084E04DDFA4C0843609F064C02EDFB82E15
:103DF0002CDFA82E992429DF853411F431E0932E8D
:103E0000C0E0D0E0CA15DB0550F400E610E01DDF8D
:103E1000F80181938F012196CA15DB05C0F315DFE8
:103E2000803209F086CF9920A9F0C0E0D0E0CA1511
:103E3000DB0508F03DC000E610E0F80161918F015C
:103E4000C6012ADF0894C11CD11C2196CA15DB05C6
:103E5000A0F32EC0CC0CDD1CEE1CFF1CA0FE03C08A
:103E60000894A11CB11CF894E199FECF1127EC2D08
:103E7000FD2DAA2DBB2DC0E6D0E0103021F483E04B
:103E800059D081E157D00990199081E053D0139512
:103E9000103428F0112785E04DD081E14BD03296C7
:103EA000129709F0EACF103011F01296F3CF1124D7
:103EB00084E136C0843739F5C8DEB82EC6DEA82EB8
:103EC000C4DE853419F491E0992E05C09924CC0CF8
:103ED000DD1CEE1CFF1CB9DE803209F02ACF84E124
:103EE000A2DEC0E0D0E0CA15DB05D8F4992019F0B5
:103EF000C601DDDE02C0F601849195DE0894C11C86
:103F0000D11C2196F0CF853779F49FDE803209F0FD
:103F100010CF84E188DE8EE186DE84E984DE83E0F2
:103F200082DE80E180DE05CF863709F002CF80E0B7
:103F300099DEFFCE9091570090FDFCCF8093570003
:043F4000E895089563
:0400000300003CBEFF
:00000001FF
